:100000004CEF03F00000000000EF00F000000000E3
:0A0010000000000000000000F3D71C
:0C001C00000000000000000000001200C6
:10002800240E0C6EB50E0D6E0D2EFED70C2EFCD7C1
:06003800000000001200B0
:0A003E00530E0D6E0D2EFED71200BA
:10004800010161BF02D08B9601D08B8661BD02D0C1
:100058008B9401D08B8461BB02D08B9201D08B82B0
:1000680061B902D08B9001D08B80000184B102D09D
:10007800898801D08998898ACDDF899A010161B779
:1000880002D08B9601D08B8661B502D08B9401D0BB
:100098008B8461B302D08B9201D08B8261B102D084
:1000A8008B9001D08B80000184B102D0898801D067
:1000B8008998898AAFDF899A84A102D0B1DF01D0FB
:0400C800BADF120089
:1000CC00AECF02F0ABA202D0AB98AB8802C001F06D
:0600DC0001C000F012005B
:0E00E200000E9EBA010E016E01C000F0120069
:0C00F000240E0D6E0D2EFED70000120035
:1000FC0001015E51010A03E1800E5E6F14D05E5166
:10010C00020A03E1C00E5E6F0ED05E51030A03E1DA
:10011C00940E5E6F08D05E51040A03E1D40E5E6F3C
:10012C0002D0800E5E6F5F05006E5E51002600C02F
:10013C005EF10001848100C061F180DF849160C1B7
:08014C0061F17CDF84811200E7
:0E015400000184915EC161F175DF84811200AB
:10016200086A096A100E0C6E01340836093604500A
:10017200085E0550D8A0053C095ED8B007D00450EF
:1001820008260550D8B0053C0926D890003601361D
:060192000C2EEAD712005A
:100198000900F5CFE6FF0006FBE10106F9E11200D0
:1001A8009CDF0050010AFCE18DDF00C058F158C106
:0401B80000F0120041
:1001BC00700E0101616F42DF01015A6BBC0E5A25B2
:1001CC00F66E120EF76E000EF722000EF86E000E91
:1001DC00F8220900F5CF5EF1B7DF01015A51070A89
:1001EC0002E05A2BEBD7020E616F28DF58C15EF18B
:0E01FC0059C15FF1060E0101606F7ADF12003B
:10020A00500E0101616F1BDF01015A6B8C0E5A25DA
:10021A00F66E120EF76E000EF722000EF86E000E42
:10022A00F8220900F5CF5EF190DF01015A51070A61
:10023A0002E05A2BEBD7020E616F01DF58C15EF163
:0E024A0059C15FF1020E0101606F53DF120017
:10025800680E0101616FF4DE01015A6B940E5A2594
:10026800F66E120EF76E000EF722000EF86E000EF4
:10027800F8220900F5CF5EF169DF01015A51070A3A
:1002880002E05A2BEBD7020E616FDADE58C15EF13D
:0E02980059C15FF1050E0101606F2CDF1200ED
:1002A600929A92989490949294949496899A899812
:1002B6008B968B948B928B90B4DEB3DEB2DE8B8200
:1002C6008B80898AA8DE899AACDE898AA4DE899A1F
:1002D600A8DE898AA0DE899AA4DE8B90898A9BDEB5
:1002E600899A9FDE898A97DE899A8B928B86898A7C
:1002F60092DE899A96DE8B968B80898A8CDE899A25
:100306008B90898A88DE899A8CDE898A84DE899A2E
:100316008B80898A80DE899A84DE8B90898A7BDE4F
:10032600899A8B868B848B828B80898A74DE899AE4
:0803360078DE00018481120051
:10033E00480E0101616F81DE01015A6BAC0E5A2528
:10034E00F66E120EF76E000EF722000EF86E000E0D
:10035E00F8220900F5CF5EF1F6DE01015A51070AC7
:10036E0002E05A2BEBD7020E616F67DE58C15EF1C9
:0E037E0059C15FF1010E0101606FB9DE12007E
:10038C00580E0101616F5ADE01015A6B9C0E5A2501
:10039C00F66E120EF76E000EF722000EF86E000EBF
:1003AC00F8220900F5CF5EF1CFDE01015A51070AA0
:1003BC0002E05A2BEBD7020E616F40DE58C15EF1A2
:0E03CC0059C15FF1030E0101606F92DE120055
:1003DA00FF0E0001856FFF0E866FFF0E876FFF0EFF
:0E03EA00886FC26A070EC012C08EC280120059
:1003F800600E0101616F24DE01015A6BA40E5A25BB
:10040800F66E120EF76E000EF722000EF86E000E52
:10041800F8220900F5CF5EF199DE01015A51070A69
:1004280002E05A2BEBD7020E616F0ADE58C15EF16B
:0E04380059C15FF1040E0101606F5CDE12001D
:10044600400E0101616FFDDD01015A6BB40E5A25A4
:10045600F66E120EF76E000EF722000EF86E000E04
:10046600F8220900F5CF5EF172DE01015A51070A42
:1004760002E05A2BEBD7020E616FE3DD58C15EF145
:0C04860059C15FF10101606B36DE12000D
:10049200C26A070EC012C08E58C100F0003600902A
:1004A200003600900050C212C28021DEC282C2A277
:1004B20002D00000FCD7C4CF01F0006A00C059F19D
:1004C20001C05AF1C35001015913000E5A13C290D0
:0A04D20059C100F05AC101F01200F8
:1004DC005AC1E1FF5BC1E2FF300EE66E300EE66EF4
:1004EC00300EE66E300EE66E300EE66EE66A040EE8
:1004FC0001015A255C6F000E5B215D6F000E5919CE
:10050C0002E1000E581927E00A0E046E000E056E6B
:10051C0058C100F059C101F01EDE08C000F009C03E
:10052C0001F0300E00265CC1E1FF5DC1E2FF00C0AE
:10053C00E6FF0A0E046E000E056E58C100F059C19C
:10054C0001F009DE00C058F101C059F1010E5C5FE9
:08055C00000E5D5BD3D7120015
:10056400FF0E0001896FFF0E8A6FFF0E8B6FFF0E67
:100574008C6FCC0E956F000E966F000E976F000E69
:10058400986FE20E916F000E926F000E936F000E43
:10059400946FFF0E8D6FFF0E8E6F000E8F6F000E27
:1005A400906FAC8A900EAB6E948E949C9EAA03D0EE
:0805B400AECF00F0FBD71200EE
:1005BC0001015851010A03E1800E586F14D05851B3
:1005CC00020A03E1C00E586F0ED05851030A03E122
:1005DC00940E586F08D05851040A03E1D40E586F8A
:1005EC0002D0800E586F5905006E5851002600C07D
:1005FC0058F100C061F122DD849101015C6B5C510A
:10060C005A25E96E000E5B21EA6EEE50000A0CE0F2
:10061C005C515A25E96E000E5B21EA6EEECF5EF15D
:0E062C0093DD01015C2BEBD7000184811200ED
:10063A000001CE6BCE510101595D1FE30001CE517D
:10064A0001015A25E16E000E5B21E26E0001CE51D6
:10065A0001015825006ECF0EE96E000EEA6E0050B9
:10066A00E926D8B0EA2AEECFE6FF0001CE51010111
:10067A00591903E00001CE2BDDD7010159515A2542
:0E068A00E16E000E5B21E26E000EE66E1200C5
:10069800B886020EB06E080EAF6EAC845FDF030E34
:1006A8000B6E8A0E0C6E550E0D6E0D2EFED70C2E8F
:1006B800FCD70B2EFAD7000000009498948A010EFC
:1006C800C26E87DE8B88200E0101346F520E356FA3
:1006D800650E366F630E376F650E386F700E396FA3
:1006E800740E3A6F650E3B6F750E3C6F720E3D6F60
:1006F800200E3E6F470E3F6F500E406F530E416FF6
:10070800200E426F200E436F446B200E236F520E53
:10071800246F450E256F590E266F410E276F580E10
:10072800286F200E296F520E2A6F590E2B6F470E15
:100738002C6F320E2D6F350E2E6F440E2F6F490E13
:10074800306F200E316F200E326F336B4C0E126FEC
:10075800650E136F630E146F740E156F750E166F9A
:10076800720E176F650E186F200E196F540E1A6FE0
:10077800720E1B6F610E1C6F6D0E1D6F650E1E6F66
:10078800730E1F6F200E206F200E216F226B4E0EEE
:100798005A6E4D0E5B6E450E5C6E410E5D6E200E00
:1007A8005E6E650E5F6E6E0E606E200E616E630E7D
:1007B800626E6F0E636E750E646E720E656E730EEA
:1007C800666E2E0E676E2E0E686E2E0E696E6A6A43
:1007D80066DD010E0101616F33DC0C0E0101616FF2
:1007E8002FDC010E0101586F010E596F340E5A6F3C
:1007F800010E5B6FDFDE010E0101586F030E596FAA
:100808009ADD010E0101586F060E596F18DE020EAF
:100818000101586F010E596F230E5A6F010E5B6F5D
:10082800C9DE7F0E0B6ED40E0C6E310E0D6E0D2EC2
:10083800FED70C2EFCD70B2EFAD700000000010EB5
:100848000101586F010E596F120E5A6F010E5B6F3E
:10085800B1DE020E0101586F010E596F5A0E5A6F20
:10086800000E5B6FA7DE4D0E0B6E190E0C6E4F0E51
:100878000D6E0D2EFED70C2EFCD70B2EFAD70000CE
:1008880000008B98010E596E560E586E6B6A010E59
:10089800786E300E6D6E300E6E6E6F6A6C6A80DC2C
:1008A80000C0CEF00050240A01E0F9D70001CE6B59
:1008B800CF0E0101566F000E576F0001CE51010196
:1008C8005627D8B0572B6CDC56C1E1FF57C1E2FF61
:1008D80000C0E6FFCF0EE96E000EEA6E0001CE51B1
:1008E800E926D8B0EA2AEE502A0A02E1CE6B01D0F6
:1008F800CE2BCE51000AFF0ED8A4000E016ECE51A9
:10090800420AFF0ED8A4000E006E0150001201E149
:10091800CFD75950010AD8A481D0D151520AFF0E1D
:10092800D8A4000E016ED2514D0AFF0ED8A4000EB5
:10093800006E00500116D351430AFF0ED8A4000ED2
:10094800006E015000166AE0020E596E010E6B6EC1
:1009580058C0CEF0DFC058F0DF51CE1905E0010EC7
:100968000101616F24EC00F05850410A57E18B886F
:10097800060E0101586F060E596F2B0E5A6F000EA6
:100988005B6F57DE120E586F020E596F200E5A6FAA
:10099800000E5B6F4EDE140E586F020E596F150E67
:1009A8005A6F000E5B6F45DE170E586F040E596FB5
:1009B800360E5A6F000E5B6F3CDEECC057F01F0E10
:1009C800586F030E596F4C0E5A6F000E5B6F31DE75
:1009D800220E586F020E596F410E5A6F000E5B6F50
:1009E80028DE250E586F040E596F790E5A6F000EC7
:1009F8005B6F1FDEFAC0AFF02D0E586F040E596FF3
:100A0800A40E5A6F000E5B6F14DE340E586F060E7C
:100A1800596F990E5A6F000E5B6F0BDE5950020A20
:100A28003CE10001D151470AFF0ED8A4000E016E27
:100A3800D251470AFF0ED8A4000E006E00500116CE
:100A4800D351410AFF0ED8A4000E006E01500016C3
:100A580024E0010E596E010E6B6E5850410A1DE1DB
:100A68008B882D0E0101586F020E596F6D0E5A6F4B
:100A7800000E5B6FDEDD300E586F040E596FB00E3E
:100A88005A6F000E5B6FD5DD350E586F030E596F28
:100A9800C30E5A6F000E5B6FCCDD0101586BF5DC9D
:100AA80000C002F001C003F003320232039E02C00C
:100AB800C1F003C0C2F002C058F103C059F1BB0E27
:100AC8005A6F000E5B6F06DD6B50010AD8A4D7D3AE
:100AD80082BA18D0782A070E0B6E580E0C6E590E73
:100AE8000D6E0D2EFED70C2EFCD70B2EFAD700005C
:100AF80000007850050A02E1010E786E010E616F60
:100B080024EC00F05850560AD8A4F1D08B98010E66
:100B18000101586F010E596F540E456F720E466FE2
:100B2800610E476F6D0E486F650E496F730E4A6F01
:100B3800200E4B6F690E4C6F6E0E4D6F760E4E6F1A
:100B4800610E4F6F6C0E506F690E516F640E526FCD
:100B5800650E536F730E546F556B450E5A6F010E29
:100B68005B6F28DD020E0101586F010E596F200ED0
:100B7800456F200E466F200E476F200E486F200EDF
:100B8800496F200E4A6F200E4B6F200E4C6F200EBF
:100B98004D6F200E4E6F200E4F6F200E506F200E9F
:100BA800516F200E526F200E536F200E546F556BED
:100BB800450E5A6F010E5B6FFDDC6C2A020E0101B7
:100BC800586F6CC059F1DEEC00F06C50100AD8B4C4
:100BD8006C6A82BA8BD08B88010E0101586F010EA6
:100BE800596F420E456F610E466F740E476F740E53
:100BF800486F650E496F720E4A6F690E4B6F650E2E
:100C08004C6F3A0E4D6F200E4E6F4F6B450E5A6F5C
:100C1800010E5B6FCFDC010E01015E6F0B0E5F6F83
:100C2800BDC060F17EEC00F0010E0101586F0C0EA2
:100C3800596F2CEC01F0010E01015E6F0D0E5F6F14
:100C4800BEC060F17EEC00F0010E01015E6F0E0E79
:100C58005F6FBFC060F17EEC00F0010E0101586FBC
:100C68000F0E596F200E456F560E466F476B450E97
:100C78005A6F010E5B6F9EDC020E0101586F010E68
:100C8800596F200E456F200E466F200E476F200EBD
:100C9800486F200E496F200E4A6F200E4B6F200EB2
:100CA8004C6F200E4D6F200E4E6F200E4F6F200E92
:100CB800506F200E516F200E526F200E536F200E72
:100CC800546F556B450E5A6F010E5B6F73DC330E14
:100CD8000B6EBB0E0C6EDF0E0D6E0D2EFED70C2E9E
:100CE800FCD70B2EFAD7000000008B98C7D278509B
:100CF800010AD8A49FD0010E0101586F010E596F47
:100D08004C0E456F410E466F540E476F3A0E486FB2
:100D1800200E496F4A6B450E5A6F010E5B6F4ADC15
:100D2800010E0101586F060E596F200E5A6F000E02
:100D38005B6F40DC010E01015E6F080E5F6FDF0E16
:100D4800606F7EEC00F0010E0101586F090E596FBB
:100D5800150E5A6F000E5B6F2DDC010E01015E6FE0
:100D68000B0E5F6F2E0E606F7EEC00F0010E01011E
:100D7800586F0C0E596F360E5A6F000E5B6F1ADCE7
:100D8800010E01015E6F100E5F6F57C060F17EECBF
:100D980000F0020E0101586F010E596F4C0E456F9D
:100DA8004F0E466F4E0E476F3A0E486F496B450E11
:100DB8005A6F010E5B6FDEEC02F0020E0101586FF4
:100DC800050E596F4C0E5A6F000E5B6FDEEC02F089
:100DD800020E01015E6F080E5F6FDF0E606F7EEC22
:100DE80000F0020E0101586F090E596F410E5A6F3B
:100DF800000E5B6FDEEC02F0020E01015E6F0B0E5F
:100E08005F6F2E0E606F7EEC00F0020E0101586FCE
:100E18000C0E596F790E5A6F000E5B6FDEEC02F004
:100E2800020E01015E6F100E5F6FAFC060F17EECC5
:100E380000F024D27850020AD8A487D0010E01010C
:100E4800586F010E596F410E456F4C0E466F540E88
:100E5800476F3A0E486F200E496F4A6B450E5A6F1E
:100E6800010E5B6FDEEC02F0010E0101586F060EF9
:100E7800596FC30E5A6F000E5B6FDEEC02F0010E65
:100E88000101586F090E596F200E456F6D0E466FA0
:100E9800650E476F740E486F720E496F650E4A6F84
:100EA800730E4B6F200E4C6F4D6B450E5A6F010E33
:100EB8005B6FDEEC02F0010E0101586F0B0E596FEB
:100EC800C6EC01F0020E0101586F010E596F560E63
:100ED800456F490E466F540E476F3A0E486F200E05
:100EE800496F4A6B450E5A6F010E5B6FDEEC02F0DC
:100EF800020E0101586F060E596FA40E5A6F000EAC
:100F08005B6FDEEC02F0020E0101586F070E596F9D
:100F18002CEC01F0020E0101586F0A0E596F200ED9
:100F2800456F6E0E466F6F0E476F650E486F750EF4
:100F3800496F640E4A6F730E4B6F4C6B450E5A6FB8
:100F4800010E5B6FDEEC02F099D17850030AD8A449
:100F5800F0D0010E0101586F010E596F4C0E456F0C
:100F6800650E466F3A0E476F200E486F496B450E67
:100F78005A6F010E5B6FDEEC02F0010E01015E6F2D
:100F8800050E5F6F99C060F17EEC00F0010E010163
:100F98005E6F060E5F6F9AC060F17EEC00F0010E86
:100FA8000101586F070E596FFCEC01F0010E0101A9
:100FB8005E6F080E5F6F9BC060F17EEC00F0010E63
:100FC80001015E6F090E5F6F9CC060F17EEC00F05E
:100FD800010E0101586F0A0E596FFCEC01F0010E69
:100FE8000101586F0B0E596F320E456F300E466F68
:100FF800476B450E5A6F010E5B6FDEEC02F0010E77
:1010080001015E6F0D0E5F6F9DC060F17EEC00F018
:10101800010E01015E6F0E0E5F6F9EC060F17EECE7
:1010280000F0010E0101586F0F0E596F200E456F29
:10103800200E466F476B450E5A6F010E5B6FDEEC54
:1010480002F0020E0101586F010E596F410E456FF3
:10105800200E466F3A0E476F200E486F496B450EBB
:101068005A6F010E5B6FDEEC02F0020E0101586F41
:10107800010E596F05EC01F0020E01015E6F050EBD
:101088005F6F2BC060F17EEC00F0020E01015E6F15
:10109800060E5F6F2CC060F17EEC00F0020E0101BD
:1010A8005E6F070E5F6F3A0E606F7EEC00F0020E07
:1010B80001015E6F080E5F6F2DC060F17EEC00F0DD
:1010C800020E01015E6F090E5F6F2EC060F17EECAB
:1010D80000F0020E01015E6F0A0E5F6F3A0E606F3C
:1010E8007EEC00F0020E01015E6F0B0E5F6F2FC0E9
:1010F80060F17EEC00F0020E01015E6F0C0E5F6F76
:1011080030C060F17EEC00F0020E0101586F0D0E48
:10111800596F200E456F550E466F540E476F430E9C
:10112800486F496B450E5A6F010E5B6FDEEC02F09B
:10113800A5D07850040AD8A4A1D0010E0101586F97
:10114800010E596F530E456F410E466F540E476F8F
:101158003A0E486F496B450E5A6F010E5B6FDEEC15
:1011680002F0010E0101586F050E596F6D0E5A6F8E
:10117800000E5B6FDEEC02F0010E0101586F080EE5
:10118800596F420E456F410E466F540E476F3A0E27
:10119800486F496B450E5A6F010E5B6FDEEC02F02B
:1011A800010E01015E6F0C0E5F6FBDC060F17EEC39
:1011B80000F0010E0101586F0D0E596F2CEC01F073
:1011C800010E01015E6F0E0E5F6FBEC060F17EEC16
:1011D80000F0010E01015E6F0F0E5F6FBFC060F17E
:1011E8007EEC00F0010E01015E6F100E5F6F560E6F
:1011F800606F7EEC00F0020E0101586F010E596F0E
:10120800480E456F440E466F4F0E476F500E486F9D
:101218003A0E496F200E4A6F4B6B450E5A6F010EFE
:101228005B6FDEEC02F0020E0101586F070E596F7A
:10123800B00E5A6F000E5B6FDEEC02F0020E010179
:10124800586F080E596F2CEC01F0020E0101586F0F
:101258000B0E596F200E456F200E466F200E476FFC
:10126800200E486F200E496F200E4A6F4B6B450EBB
:101278005A6F010E5B6FDEEC02F000D06B6A53EF21
:0412880004F0FFD798
:08128C0008040E010F110F0010
:0812940000000000000C04083A
:08129C0008040E111F100E00E2
:0812A4000000000E0000000034
:0812AC0002040E111F100E00D8
:0812B40000001E11111E1010B4
:0812BC00181C1E1F1F1E1C1848
:020000040030CA
:0D000100021F1EFF8381FF0FC00FE00F40A4
:00000001FF
